:020000040000FA
:42000000FFFF62F73300FFFFFFFFFFFFFFFFFFFFFFFFFFFFFFFFFFFFFFFFFFFFFFFFFFFFFFFFFFFFFFFFFFFFFFFFFFFFFFFFFFFFFFFFFFFFFFFFFFFFFFFFFFFFFFFFFFFFFFFF70
:42004200A00C9481325006CA4019005360064C81A9325506CA401928034C80613001000000000006984013001324830C900132400618061360022002648001300006C000D4FE86
:420084000015A00254800A50012A800A50012A4005B4800A50012A4005A8002DA00200000000000950012A800E780117E0025C800BD0022A400550012A400248000920013CFE56
:4200C6000004800010000240000800024000080001300002400008000100000000000000000000000000000000000000000000000000000000000000000000000000000010FC48
:42010800000000000000000000000000000000000000000000000000000000000000000000000000000000000000000000000000000000000000000000000000000000003CFE7B
:42014A000001200004800010000200080001200004848000108002400000000000000000000000000000000008080000000000000000000000000000000000000000000074FD38
:42018C000001080004800220000200424480081001118402100000800000000000000000000000000000000000000000000000000000000000000000000000000000000070FECC
:4201CE000000000000000000000000000000000000000000000000000000000000000000000000840000000000000000000006020000000000000000000000000200000074FEEF
:420210000000000000000000000000000000000000000000000000000000000000000000000000000000000000000000000006000000000000000000000000000000000018FC92
:4202520000000000000000000000000000000000000000000000000000000000000000000000F00000000000000000000080010000000000000000000000800100000000D4FEA6
:4202940000000000000000000000000000000000000000000000000000000000000000000000D02200000000000000000080000000000000000000000000800000000000C4FE74
:4202D600000000000000000000000000000000000000000000000000000000000000000000000004000000000000000000001002000000000000000000000016010000002CFF8E
:4203180000000000000000000000000000000000000000000000000000000000000000000000F0400000000000000000008001000000000000000000000080070000000094FCDB
:42035A000000000000000000000000000000000000000000000000000000000000000000000000000000000000000000000000000000000000000000000000060000000078FCE7
:42039C0000000000000000000000000000000000000000000000000000000000000000000000C01000000000000000000080A0000000000000000000000080060000000000FDAC
:4203DE0000000000000000000000000000000000000000000000000000000000000000000000C082000000000000000000800000000000000000000000000000000000005EFEBF
:42042000000000000000000000000000000000000000000000000000000000000000000000000000000000000000000000000000000000000000000000000000000000003CFE60
:4204620000000000000000000000000000000000000000000000000000000000000000000000F00000000000000000000000000000000000000000000000000000000000CCFE9E
:4204A4000800000000000000000000000000000000000000000000000000000000000000000010100000000000000000000000000000000000000000000000000000008025FE4B
:4204E60000000000000000000000000000000000000000000000000000000000000000000000000000000000000000000000100000000000000000000000000000000080A4FEA2
:4205280000000000000000000000000000000000000000000000000000000000000000000000F0000000000000000000008001020000000000000000000000000000000054FDCD
:42056A0004000000000000000000000000000000000000000000000000000000000000000000000000000000000000000000060000000000000000000000000000000080C1FD07
:4205AC0000000000000000000000000000000000000000000000000000000000000000000000D00000000000000000000000160100000000000000000000000000000000D8FD51
:4205EE0000000000000000000000000000000000000000000000000000000000000000000000C0221A00000000000000000006020000000000000000000000000000000058FF70
:420630000000000000000000000000000000000000000000000000000000000000000000000000000000000000000000000006000000000000000000000000000000000018FC6E
:4206720000000000000000000000000000000000000000000000000000000000000000000000F0001E04000000000000008007000000000000000000000000000000000094FC1D
:4206B4000400000000000000000000000000000000000000000000000000000000000000000010441A00000000000000008006000000000000000000000000000000000031FCDF
:4206F6000C000000000000000000000000000000000000000000000000000000000000000000000098000000000000000000060000000000000000000000000000000000D0FD4B
:4207380000000000000000000000000000000000000000000000000000000000000000000000F0001E08000000000000008007000000000000000000000000000000000098FC4E
:42077A000800000000000000000000000000000000000000000000000000000000000000000000001804000000000000000006000000000000000000000000000000008094FD02
:4207BC0000000000000000000000000000000000000000000000000000000000000000000000C0009800000000000000008006000000000000000000000000000000000058FDC8
:4207FE0000000000000000000000000000000000000000000000000000000000000000000000100000000000000000000080000000000000000000000000000002000000A6FC85
:42084000000000000000000000000000000000000000000000000000000000000000000000000000000000000000000000000000000000000000000000000000000000003CFE3C
:420882000000000000000000000000000000000000000000000000000000000000000000000030000000000000000000008001000000000000000000000080010000000014FEF0
:4208C400080000000000000000000000000000000000000000000000000000000000000000001000000000000000000000800000000000000000000000008000000000803DFF1E
:4209060000000000000000000000000000000000000000000000000000000000000000000000C0440000000000000000000016020000000000000000000000460100008050FC80
:4209480000000000000000000000000000000000000000000000000000000000000000000000F00000000000000000000080070000000000000000000000800700000000B4FEBD
:42098A0004000000000000000000000000000000000000000000000000000000000000000000C0000000000000000000000000000000000000000000000000060000008061FD83
:4209CC0000000000000000000000000000000000000000000000000000000000000000000000C00000000000000000000000A0000000000000000000000080060000000098FC6F
:420A0E0000000000000000000000000000000000000000000000000000000000000000000000D0000000000000000000008000000000000000000000000000000200000066FCF2
:420A500000000000000000000000000000000000000000000000000000000000000000000000C00000000000000000000000000000000000000000000000000000000000FCFEAA
:420A920000000000000000000000000000000000000000000000000000000000000000000000000000000000000000000000000000000000000000000000800100000000BCFFE6
:420AD4000400000000000000000000000000000000000000000000000000000000000000000000000000000000000000000000000000000000000000000080000000008065FF78
:420B16000C00000000000000000000000000000000000000000000000000000000000000000000040000000000000000000016020000000000000000000000060100008050FCA2
:420B58000000000000000000000000000000000000000000000000000000000000000000000030400000000000000000008007000000000000000000000080070000000070FE6F
:420B9A000800000000000000000000000000000000000000000000000000000000000000000000000000000000000000000000000000000000000000000000060000008061FD2D
:420BDC0000000000000000000000000000000000000000000000000000000000000000000000004200000000000000000000A000000000000000000000008006000000005CFE15
:420C1E0000000000000000000000000000000000000000000000000000000000000000000000102000000000000000000080000000000000000000000000001604000000B2FD1B
:420C6000000000000000000000000000000000000000000000000000000000000000000000000000000000000000000000000000000000000000000000000000000000003CFE18
:420CA20000000000000000000000000000000000000000000000000000000000000000000000000000000000000000000000000000000000000000000000800700000000F8FD94
:420CE40008000000000000000000000000000000000000000000000000000000000000000000008200000000000000000000000000000000000000000000802002000080ADFF76
:420D26000000000000000000000000000000000000000000000000000000000000000000000000240000000000000000000040000000000000000000000000000000008090FC1B
:420D68000000000000000000000000000000000000000000000000000000000000000000000030000000000000000000008001040000000000000000000080070000000014FCFD
:420DAA000400000000000000000000000000000000000000000000000000000000000000000080000000000000000000000006000000000000000000000000000000008041FDBF
:420DEC0000000000000000000000000000000000000000000000000000000000000000000000002800000000000000000000160100000000000000000000000600000000E4FD9F
:420E2E000000000000000000000000000000000000000000000000000000000000000000000000220200000000000000008000000000000000000000000000160400000082FF43
:420E70000000000000000000000000000000000000000000000000000000000000000000000000000000000000000000000006000000000000000000000000000000000018FC26
:420EB2000000000000000000000000000000000000000000000000000000000000000000000030000600000000000000008001000000000000000000000080070200000010FCB2
:420EF40004000000000000000000000000000000000000000000000000000000000000000000100002000000000000000080A000000000000000000000008010000000806DFE0B
:420F36000C000000000000000000000000000000000000000000000000000000000000000000C0089800000000000000000026000000000000000000000000000000008030FD3A
:420F780000000000000000000000000000000000000000000000000000000000000000000000F0201E0800000000000000800701000000000000000000008007000000007CFC7A
:420FBA0008000000000000000000000000000000000000000000000000000000000000000000C0001800000000000000000006020000000000000000000000000000008041FE4E
:420FFC0000000000000000000000000000000000000000000000000000000000000000000000C0001800000000000000008016000000000000000000000000060000000084FFBC
:42103E000000000000000000000000000000000000000000000000000000000000000000000010000200000000000000008000000000000000000000000000160400000090FD37
:42108000000000000000000000000000000000000000000000000000000000000000000000000000000000000000000000000000000000000000000000000000000000003CFEF4
:4210C2000000000000000000000000000000000000000000000000000000000000000000000030000600000000000000008007000000000000000000000080070000000014FE96
:4211040008000000000000000000000000000000000000000000000000000000000000000000100002000000000000000080200100000000000000000000802004000000D5FC79
:4211460000000000000000000000000000000000000000000000000000000000000000000000C004180500000000000000001000000000000000000000000000000000003CFE3C
:4211880000000000000000000000000000000000000000000000000000000000000000000000F0201E00000000000000008007020000000000000000000080070000000074FF74
:4211CA0004000000000000000000000000000000000000000000000000000000000000000000C00018000000000000000000000000000000000000000000000000000080B4FFD4
:42120C0000000000000000000000000000000000000000000000000000000000000000000000C00018000000000000000080060400000000000000000000000600000000D0FF69
:42124E00000000000000000000000000000000000000000000000000000000000000000000000000000000000000000000000400000000000000000000000004000000005EFCFC
:42129000200004800010000240000800012000048000100002400008000120000400000000000000024000080001200004000010000240000800012000040000100002002CFCD2
:4212D20000000000000000000000000000000000000000000000000000000000000000000000800000000000000000000000000000000000000000000000000000000000BCFEA0
:4213140024000480001000024000080001200004800010000240000800012000040000000000100002400008000120000480001000024000080001200004800010000280EDFDF7
:421356000C00000000000000000000000000000000000000000000000000000000000000000000000000000000000000000004000000000000000000000000040000008034FE8F
:42139800200004800010000240000800012000048000100002400008000120000400000000000000004000080001200004000010000240000800012000040000100002000CFCEB
:4213DA0008000000000000000000000000000000000000000000000000000000000000000000800010000000000000000000000000000000000000000000000000000080A5FE16
:42141C002000048000100002400008000120000480001000024000080001200004000000000010000240000800012000048000100002400008000120000480001000020034FC2C
:42145E00000000000000000000000000000000000000000000000000000000000000000000000000000000000000000000000000000000000000000000000000000000003CFE12
:4214A000000000000000000000000000000000000000000000000000000000000000000000000000000000000000000000000000000000000000000000000000000000003CFED0
:4214E200000000000000000000000000000000000000000000000000000000000000000000000000000000000000000000000000000000000000000000000000000000003CFE8E
:4215240000000000000000000000000000000000000000000000000000000000000000000000000000000000000000000000000000000000000000000000000000000080B4FE53
:42156600000000000000000000000000000000000000000000000000000000000000000000000000000000000000000000000000000000000000000000000000000000003CFE09
:4215A80000000000000000000000000000000000000000000000000000000000000000000000000100000000000000000000000000000000000000000000000802000040D0FFE7
:4215EA00000000000000000000000000000000000000000000000000000000000000000000000000000000000000000000000000000000000000000000000000000000003CFE85
:42162C00000000000000000000000000000000000000000000000000000000000000000000000000000000000000000000000000000000000000000000000000000000003CFE42
:42166E00000000000000000000000000000000000000000000000000000000000000000000000000000000000000000000000000000000000000000000000000000000003CFE00
:4216B00000000000000000000000000000000000000000000000000000000000000000000000000000000000000000000080000000000000000000000000000000000000B4FEC6
:4216F200000000000000000000000000000000000000000000000000000000000000000000000000000000000000000000000000000000000000000000000002000000003CFC7C
:4217340000000000000000000000000000000000000000000000000000000000000000000000000000000000000000000000000000000000000000000000000000000080B4FE41
:42177600000000000000000000000000000000000000000000000000000000000000000000000000000000000000000000000000000000000000000000000000010010003CFFE5
:4217B800000000000000000000000000000000000000000000000000000000000000000000000000000000000000000000000000000000000000000000000000000000003CFEB5
:4217FA00000000000000000000000000000000000000000000000000000000000000000000000014080000000000000000000000000000000000000000000000020004008CFF00
:42183C0000000000008000000002000800000000000000000000020000000000000000000000000000000100000000000000000200000000000000000000000200000000BCFD20
:42187E00000000000000000000000000000000000000000000000000000000000000000000000000000002000000000000000000000000000000000000000002000000003CFEEA
:4218C0000000000000800000000200400000000000000000000002000000000000000000000000000000000000000000000000000000000000000000000000000000000030FCF6
:42190200000000000000000000000000000000000000000000000000000000000000000000000000000000000000000000000000000000000000000000000000000000003CFE69
:42194400000000000000000000000000000000000000000000000000000000000000000000000000000000000000000000000000000000000000000000000000000000003CFE27
:42198600000000000000000000000000000000000000000000000000000000000000000000000000000000000000000000000000000000000000000000000000000000003CFEE5
:4219C800000000000000000000000000000000000000000000000000000000000000000000000000000000000000000000000000000000000000000000000000000000003CFEA3
:421A0A00000000000000000000000000000000000000000000000000000000000000000000001000000000000000000000000000000000000000000000000000000000002CFE60
:421A4C00000000000000000000000000000000000000000000000000000000000000000000000000000000000000000000000000000000000000000000000000000000003CFE1E
:421A8E00000000000000000000000000000000000000000000000000000000000000000000000000000000000000000000000000000000000000000000000000000000001EFCFC
:421AD000000000000000000000000000000000000000000000000000000000000000000000000000000000000000000000000000000000000000000000000000000000003CFE9A
:421B1200000000000000000000000000000000000000000000000000000000000000000000000000000000000000000000000000000000000000000000000000000000003CFE57
:421B540000000000000000000000000000000000000000000000000000000000000000000000800000000000000000000000040000000000000000000000000000000000B8FE15
:421B9600000000000000000000000000000000000000000000000000000000000000000000000000000000000000000000000000000000000000000000000000000000003CFED3
:421BD800000000000000000000000000000000000000000000000000000000000000000000000000000000000000000000000000000000000000000000000000000000002DFF9F
:421C1A00000000000000000000000000000000000000000000000000000000000000000000000000000000000000000000000200000000000000000000000000000000001CFC6E
:421C5C00000000000000000000000000000000000000000000000000000000000000000000000000000000000000000000000000000000000000000000000000000000003CFE0C
:421C9E0000000000000000000000000000000000000000000000000000000000000000000000800010000000000000000000010000000000000000000000000100000000ACFFC7
:421CE000000000000000000000000000000000000000000000000000000000000000000000000010000000000000000000000000000000000000000000000000000000002CFF87
:421D2200000000000000000000000000000000000000000000000000000000000000000000000000000000000000000000000000000000000000000000000000000000003CFE45
:421D6400000000000000000000000000000000000000000000000000000000000000000000000000000000000000000000000000000000000000000000000000000000003CFE03
:421DA6000000000000000000000000000000000000000000000000000000000000000000000000000084000000000000000002000000000000000000000000010100000088FDEE
:421DE800000000000000000000000000000000000000000000000000000000000000000000000000000000000000000000000001000000000000000000000000000000002DFE8D
:421E2A00000000000000000000000000000000000000000000000000000000000000000000000000008C0000000000000000010500000000000000000000000102000000C4FF1E
:421E6C000000000000000000000000000000000000000000000000000000000000000000000000008805002010000000000005020000000000000000000000000100000034FE3D
:421EAE0000000000000000000000000000000000000000000000000000000000000000000000000008040010200000000000000000000000000000000000000002000000B8FFFD
:421EF000000000000000000000000000000000000000000000000000000000000000000000000000000000000000000000000200000000000000000000000000000000001CFC96
:421F3200000000000000000000000000000000000000000000000000000000000000000000000000000000000000000000000000000000000000000000000000000000003CFE33
:421F7400000000000000000000000000000000000000000000000000000000000000000000000000000000000000000000000000000000000000000000000000000000003CFEF1
:421FB60004000000000000000000000000000000000000000000000000000000000000000000000000000000000000000000000200000000000000000000000000000080F4FC73
:421FF800000000000000000000000000000000000000000000000000000000000000000000004000000000000000000000000000000000000000000000000000000000007CFEED
:42203A0008000000000000000000000000000000000000000000000000000000000000000000001000000000000000000000000000000000000000000000008000000000A4FF29
:42207C00000000000000000000000000000000000000000000000000000000000000000000000000000000000000000000000000000000000000000000000000000000003CFEE8
:4220BE00000000000000000000000000000000000000000000000000000000000000000000000000000000000000000000000000000000000000000000000000000000405AFC4A
:42210000000000000000000000000000000000000000000000000000000000000000000000000000000000000000000000000000000000000000000000000000000000003CFE63
:42214200000000000000000000000000000000000000000000000000000000000000000000000000000000000000000000000000000000000000000000000000000000003CFE21
:42218400000000000000000000000000000000000000000000000000000000000000000000000020000000000000000000000000000000000000000000000000000000001CFCE1
:4221C600000000000000000000000000000000000000000000000000000000000000000000000000000000000000000000000000000000000000000000000000000000003CFE9D
:42220800000000000000000000000000000000000000000000000000000000000000000000000000000000000000000000000000000000000000000000000000000000003CFE5A
:42224A00000000000000000000000000000000000000000000000000000000000000000000000000000000000000000000000000000000000000000000000000000000003CFE18
:42228C00000000000000000000000000000000000000000000000000000000000000000000000000000000000000000000000000000000000000000000000000000000003CFED6
:4222CE00000000000000000000000000000000000000000000000000000000000000000000000000000000000000000000000000000000000000000000000000000000003CFE94
:42231000000000000000000000000000000000000000000000000000000000000000000000000000000000000000000000000000000000000000000000000000000000003CFE51
:42235200000000000000000000000000000000000000000000000000000000000000000000000000000000000000000000000000000000000000000000000000000000003CFE0F
:42239400000000000000000000000000000000000000000000000000000000000000000000000000000000000000000000000000000000000000000000000000000000003CFECD
:4223D600000000000000000000000000000000000000000000000000000000000000000000000000000000000000000000000000000000000000000000000000000000003CFE8B
:42241800000000000000000000000000000000000000000000000000000000000000000000000000000000000000000000000000000000000000000000000000000000003CFE48
:42245A00000000000000000000000000000000000000000000000000000000000000000000000000000000000000000000000000000000000000000000000000000000001EFC26
:42249C00000000000000000000000000000000000000000000000000000000000000000000000000000000000000000000000000000000000000000000000000000000003CFEC4
:4224DE00000000000000000000000000000000000000000000000000000000000000000000000000000000000000000000000000000000000000000000000000000000003CFE82
:422520000800000000000000000000000000000000000000000000000000000000000000000000000000000000000000000000000000000000000000000000000000008025FFCD
:4225620000000000000000000000000000000000000000000000000000000000000000000000000000000000000000000000000000000000000000000000000000000080B4FE05
:4225A400000000000000000000000000000000000000000000000000000000000000000000000000000000000000000000000000000000000000000000000000000000003CFEBB
:4225E60004000000000000000000000000000000000000000000000000000000000000000000000000000000000000000000000000000000000000000000000000000080E5FF4B
:42262800000000000000000000000000000000000000000000000000000000000000000000000000000000000000000000000000000000000000000000000000000000003CFE36
:42266A00000000000000000000000000000000000000000000000000000000000000000000000000000000000000000000000000000000000000000000000000000000003CFEF4
:4226AC00000000000000000000000000000000000000000000000000000000000000000000000000000000000000000000000000000000000000000000000000000000003CFEB2
:4226EE00000000000000000000000000000000000000000000000000000000000000000000000000000000000000000000000000000000000000000000000000000000003CFE70
:42273000040000000000000000000000000000000000000000000000000000000000000000000000000000000000000000000000000000000000000000000000000000006DFFF7
:422772000C000000000000000000000000000000000000000000000000000000000000000000000000000000000000000000000000000000000000000000000000000000FCFE1F
:4227B400000000000000000000000000000000000000000000000000000000000000000000000000000000000000000000000000000000000000000000000000000000003CFEA9
:4227F6000800000000000000000000000000000000000000000000000000000000000000000000000000000000000000000000000000000000000000000000000000008034FEE7
:42283800000000000000000000000000000000000000000000000000000000000000000000000000000000000000000000000000000000000000000000000000000000003CFE24
:42287A00000000000000000000000000000000000000000000000000000000000000000000000000000000000000000000000000000000000000000000000000000000003CFEE2
:4228BC00000000000000000000000000000000000000000000000000000000000000000000000000000000000000000000000000000000000000000000000000000000003CFEA0
:4228FE00000000000000000000000000000000000000000000000000000000000000000000000000000000000000000000000000000000000000000000000000000000003CFE5E
:42294000040000000000000000000000000000000000000000000000000000000000000000000000000000000000000000000000000000000000000000000000000000006DFFE5
:422982000C000000000000000000000000000000000000000000000000000000000000000000000000000000000000000000000000000000000000000000000000000000FCFE0D
:4229C400000000000000000000000000000000000000000000000000000000000000000000000000000000000000000000000000000000000000000000000000000000003CFE97
:422A06000800000000000000000000000000000000000000000000000000000000000000000000000000000000000000000000000000000000000000000000000000008034FED4
:422A4800000000000000000000000000000000000000000000000000000000000000000000000000000000000000000000000000000000000000000000000000000000003CFE12
:422A8A00000000000000000000000000000000000000000000000000000000000000000000000000000000000000000000000000000000000000000000000000000000001EFCF0
:422ACC00000000000000000000000000000000000000000000000000000000000000000000000000000000000000000000000000000000000000000000000000000000003CFE8E
:422B0E00000000000000000000000000000000000000000000000000000000000000000000000000000000000000000000000000000000000000000000000000000000003CFE4B
:422B500004000000000000000000000000000000000000000000000000000000000000000000000000000000000000000000000000000000000000000000000000000080E5FFDB
:422B92000C00000000000000000000000000000000000000000000000000000000000000000000000000000000000000000000000000000000000000000000000000008074FE03
:422BD400000000000000000000000000000000000000000000000000000000000000000000000000000000000000000000000000000000000000000000000000000000003CFE85
:422C16000800000000000000000000000000000000000000000000000000000000000000000000000000000000000000000000000000000000000000000000000000008025FFD0
:422C5800000000000000000000000000000000000000000000000000000000000000000000000000000000000000000000000000000000000000000000000000000000003CFE00
:422C9A000000000000000000000000000000000000000000000000000000000000000000000000000000000000000000000000000000000008000000000000000000000034FEBE
:422CDC00000000000000000000000000000000000000000000000000000000000000000000000000000000000000000000000000000000000000000000000000000000003CFE7C
:422D1E00000000000000000000000000000000000000000000000000000000000000000000000000000000000000000000000000000000000000000000000000000000003CFE39
:422D6000040000000000000000000000000000000000000000000000000000000000000000000000000000000000000000000000000000000000000000000000000000006DFFC1
:422DA2000C00000000000000000000000000000000000000000000000000000000000000000000000000000000000000000000000000000060080000000000000000000014FE69
:422DE4000000000000000000000000000000000000000000000000000000000000000000000000000000000000000000000000000000000078000000000000000000000044FEF3
:422E26000800000000000000000000000000000000000000000000000000000000000000000000000000000000000000000000000000000060000000000000000000008054FE30
:422E6800000000000000000000000000000000000000000000000000000000000000000000000000000000000000000000000000000000006000000000000000000000005CFE6E
:422EAA00000000000000000000000000000000000000000000000000000000000000000000000000000000000000000000000000000000000000000000000000000000003CFEAC
:422EEC00000000000000000000000000000000000000000000000000000000000000000000000000000000000000000000000000000000000000000000000000000000003CFE6A
:422F2E00000000000000000000000000000000000000000000000000000000000000000000000000000000000000000000000000000000000000000000000000000000003CFE27
:422F700004000000000000000000000000000000000000000000000000000000000000000000000000000000000000000000000000000000000000000000000000000080E5FFB7
:422FB2000C00000000000000000000000000000000000000000000000000000000000000000000000000000000000000000000000000000000000000000000000000008074FEDF
:422FF400000000000000000000000000000000000000000000000000000000000000000000000000000000000000000000000000000000000000000000000000000000003CFE61
:423036000800000000000000000000000000000000000000000000000000000000000000000000000000000000000000000000000000000000000000000000000000008025FFAC
:42307800000000000000000000000000000000000000000000000000000000000000000000000000000000000000000000000000000000000000000000000000000000003CFEDC
:4230BA00000000000000000000000000000000000000000000000000000000000000000000000000000000000000000000000000000000000000000000000000000000003CFE9A
:4230FC00000000000000000000000000000000000000000000000000000000000000000000000000000000000000000000000000000000000000000000000000000000003CFE58
:42313E00000000000000000000000000000000000000000000000000000000000000000000000000000000000000000000000000000000000000000000000000000000003CFE15
:4231800008000000000000000000000000000000000000000000000000000000000000000000000000000000000000000000000000000000000000000000000000000000ADFF59
:4231C200000000000000000000000000000000000000000000000000000000000000000000000000000000000000000000000000000000000000000000000000000000003CFE91
:42320400000000000000000000000000000000000000000000000000000000000000000000000000000000000000000000000000000000000000000000000000000000003CFE4E
:4232460004000000000000000000000000000000000000000000000000000000000000000000000000000000000000000000000000000000000000000000000000000080F4FED0
:42328800000000000000000000000000000000000000000000000000000000000000000000000000000000000000000000000000000000000000000000000000000000003CFECA
:4232CA00000000000000000000000000000000000000000000000000000000000000000000000000000000000000000000000000000000000000000000000000000000001EFCA8
:42330C002000048000100002400008000120000480001000024000080001200004000000000010000240000800012000048000100002400008000120000480001000020034FC1D
:42334E00000000000000000000000000000000000000000000000000000000000000000000000000000000000000000000000000000000000000000000000000000000003CFE03
:4233900024000480001000024000080001200004800010000240000800012000040000000000100002400008000120000480001000024000080001200004800010000280EDFD5B
:4233D2000C00000000000000000000000000000000000000000000000000000000000000000000000000000000000000000000000000000000000000000000000000008074FEBB
:423414002000048000100002400008000120000480001000024000080001200004000000000010000240000800012000048000100002400008000120000480001000020034FC14
:423456000800000000000000000000000000000000000000000000000000000000000000000000000000000000000000000000000000000000000000000000000000008025FF88
:423498002000048000100002400008000120000480001000024000080001200004000000000010000240000800012000048000100002400008000120000480001000020034FC90
:4234DA00000000000000000000000000000000000000000000000000000000000000000000000000000000000000000000000000000000000000000000000000000000003CFE76
:42351C00000000000000000000000000000000000000000000000000000000000000000000000000000000000000000000000000000000000000000000000000000000003CFE33
:42355E00000000000000000000000000000000000000000000000000000000000000000000000000000000000000000000000000000000000000000000000000000000003CFEF1
:4235A000000000000000000000000000000000000000000000000000000000000000000000000000000000000000000000000000000000000000000000000000000000003CFEAF
:4235E200000000000000000000000000000000000000000000000000000000000000000000000000000000000000000000000000000000000000000000000000000000003CFE6D
:42362400000000000000000000000000000000000000000000000000000000000000000000000000000000000000000000000000000000000000000000000000000000003CFE2A
:42366600000000000000000000000000000000000000000000000000000000000000000000000000000000000000000000000000000000000000000000000000000000003CFEE8
:4236A800000000000000000000000000000000000000000000000000000000000000000000000000000000000000000000000000000000000000000000000000000000003CFEA6
:4236EA00000000000000000000000000000000000000000000000000000000000000000000000000000000000000000000000000000000000000000000000000000000003CFE64
:42372C000000000000000000000000000000000000000000000000000000000000000000000000000000000000000000000000000000000000000000000000000000004078FEA5
:42376E00000000000000000000000000000000000000000000000000000000000000000000000000000000000000000000000000000000000000000000000000000000003CFEDF
:4237B0000000000000000000000000000000000000000000000000000000000000000000000000000000000000000000000000000000000000000000000000000000004078FE21
:4237F200000000000000000000000000000000000000000000000000000000000000000000000000000000000000000000000000000000000000000100000000000000002CFF69
:42383400000000000000000000000000000000000000000000000000000000000000000000000000000000000000000000000000000000000000000000000000000000003CFE18
:423876000000000000000000000000000000000000000000000000000000000000000000000000000000000000000000000000000000000000000004000000000000000038FED6
:4238B8000000000000000000000000000000000000000000000000000000000000000000000000000000000000040000000000000000000000000000000000000000000078FE54
:4238FA0000000000000000000000000000000000000000000000000000000000000000000000000000000000000800000000000000000000000000000000000000000000B4FED2
:42393C00000000000000000000000000000000000000000000000000000000000000000000000000000000000000000000000000000000000000000000000000000000003CFE0F
:42397E00000000000000000000000000000000000000000000000000000000000000000000000000000000000000000000000000000000000000000000000000000000003CFECD
:4239C000000000000000000000000000000000000000000000000000000000000000000000000000000000000000000000000000000000000000000000000000000000003CFE8B
:423A0200000000000000000000000000000000000000000000000000000000000000000000000000000000000000000000000000000000000000000000000000000000003CFE48
:423A4400000000000000000000000000000000000000000000000000000000000000000000000000000000000000000000000000000000000000000000000000000000001EFC26
:423A8600000000000000000000000000000000000000000000000000000000000000000000000000000000000000000000000000000000000000000000000000000000003CFEC4
:423AC800000000000000000000000000000000000000000000000000000000000000000000000000000000000000000000000000000000000000000000000000000000003CFE82
:423B0A00000000000000000000000000000000000000000000000000000000000000000000000000000000000000000000000000000000000000000000000000000000003CFE3F
:423B4C00000000000000000000000000000000000000000000000000000000000000000000000000000000000000000000000000000000000000000000000000000000003CFEFD
:423B8E00000000000000000000000000000000000000000000000000000000000000000000000000000000000000000000000000000000000000000000000000000000003CFEBB
:423BD000000000000000000000000000000000000000000000000000000000000000000000000000000000000000000000000000000000000000000000000000000000003CFE79
:423C1200000000000000000000000000000000000000000000000000000000000000000000000000000000000000000000000000000000000000000000000000000000003CFE36
:423C5400000000000000000000000000000000000000000000000000000000000000000000000000000000000000000000000000000000000000000000000000000000002DFF02
:423C9600000000000000000000000000000000000000000000000000000000000000000000000000000000000000000000000000000000000000000000000000000000003CFEB2
:423CD800000000000000000000000000000000000000000000000000000000000000000000000000000000000000000000000000000000000000000000000000000000003CFE70
:423D1A00000000000000000000000000000000000000000000000000000000000000000000000000000000000000000000000000000000000000000000000000000000003CFE2D
:423D5C000000000000000000000000000000000000000000000000000000000000000000000000000000000000000000000000000000000008000000000000000000000034FEEB
:423D9E00000000000000000000000000000000000000000000000000000000000000000000000000000000000000000000000000000000000000000000000000000000003CFEA9
:423DE000000000000000000000000000000000000000000000000000000000000000000000000000000000000000000000000000000000000000000000000000000000003CFE67
:423E2200000000000000000000000000000000000000000000000000000000000000000000000000000000000000000000000000000000000000000000000000000000003CFE24
:423E6400000000000000000000000000000000000000000000000000000000000000000000000000000000000000000000000000000000000000000000000000000000002DFFF0
:423EA600000000000000000000000000000000000000000000000000000000000000000000000000000000000000000000000000000000000000000000000000000000003CFEA0
:423EE800000000000000000000000000000000000000000000000000000000000000000000000000000000000000000000000200000000000010000000000000000000000CFD7D
:423F2A000000000000000000000000000000000000000000000000000000000000000000000000000000000000000000000004000000000000100000000000000000000028FF1A
:423F6C00000000000000000000000000000000000000000000000000000000000000000000000000000000000000000000000000000000000000000000000000000000003CFED9
:423FAE00000000000000000000000000000000000000000000000000000000000000000000000000000000000000000000000000000000000000000000000000000000003CFE97
:423FF000000000000000000000000000000000000000000000000000000000000000000000000000000000000000000000000000000000000000000000000000000000003CFE55
:42403200000000000000000000000000000000000000000000000000000000000000000000000000000000000000000000000000000000000000000000000000000000003CFE12
:42407400000000000000000000000000000000000000000000000000000000000000000000000000000000000000000000000000000000000000000000000000000000003CFED0
:4240B600000000000000000000000000000000000000000000000000000000000000000000000000000000000000000000000000000000000000000000000000000000003CFE8E
:4240F800000000000000000000000000000000000000000000000000000000000000000000000000000000000000000000000000000000000000000000000000000000003CFE4C
:42413A00000000000000000000000000000000000000000000000000000000000000000000000000000000000000000000000000000000000000000000000000000000003CFE09
:42417C00000000000000000000000000000000000000000000000000000000000000000000000000000000000000000000000000000000000000000000000000000000003CFEC7
:4241BE00000000000000000000000000000000000000000000000000000000000000000000000000000000000000000000000000000000000000000000000000000000003CFE85
:42420000000000000000000000000000000000000000000000000000000000000000000000000000000000000000000000000000000000000000000000000000000000003CFE42
:42424200000000000000000000000000000000000000000000000000000000000000000000000000000000000000000000000000000000000000000000000000000000003CFE00
:42428400000000000000000000000000000000000000000000000000000000000000000000000000000000000000000000000000000000000000000000000000000000003CFEBE
:4242C600000000000000000000000000000000000000000000000000000000000000000000000000000000000000000000000000000000000000000000000000020000001CFE9A
:42430800000000000000000000000000000000000000000000000000000000000000000000000000000000000000000000000000000000000000000000000000000000003CFE39
:42434A0000000000000000000000000000000000000000000000000000000000000000000000000000000000000000000000000000000000000000000000800100000000BCFFF5
:42438C0000000000000000000000000000000000000000000000000000000000000000000000000000000000000000000000000000000000000000000000800000000000BCFEB5
:4243CE00000000000000000000000000000000000000000000000000000000000000000000000000000000000000000000000000000000000000000000000046000000007CFCEF
:4244100000000000000000000000000000000000000000000000000000000000000000000000000000000000000000000000000000000000000000000000800701000000E8FDFD
:424452000000000000000000000000000000000000000000000000000000000000000000000000000000000000000000000000000000000000000000000000060000000078FCAE
:424494000000000000000000000000000000000000000000000000000000000000000000000000000000000000000000000000000000000000000000000000060000000078FC6C
:4244D600000000000000000000000000000000000000000000000000000000000000000000000000000000000000000000000000000000000000000000000046020000007EFEE0
:42451800000000000000000000000000000000000000000000000000000000000000000000000000000000000000000000000000000000000000000000000000000000003CFE27
:42455A0000000000000000000000000000000000000000000000000000000000000000000000000000000000000000000000000000000000000000000000800700000000F8FDA3
:42459C000800000000000000000000000000000000000000000000000000000000000000000000000000000000000000000000000000000000000000000080100200008095FE30
:4245DE0000000000000000000000000000000000000000000000000000000000000000000000000000000000000000000000000000000000000000000000000000000080B4FE69
:4246200000000000000000000000000000000000000000000000000000000000000000000000000000000000000000000000000000000000000000000000800700000000F8FDDC
:4246620004000000000000000000000000000000000000000000000000000000000000000000000000000000000000000000000000000000000000000000000000000080E5FFAE
:4246A40000000000000000000000000000000000000000000000000000000000000000000000000000000000000000000000000000000000000000000000800600000000F8FC5A
:4246E600000000000000000000000000000000000000000000000000000000000000000000000000000000000000000000000000000000000000000000000046020000005CFCF2
:42472800000000000000000000000000000000000000000000000000000000000000000000000000000000000000000000000000000000000000000000000000000000003CFE15
:42476A0000000000000000000000000000000000000000000000000000000000000000000000000000000000000000000000000000000000000000000000800702000000D8FDAF
:4247AC0004000000000000000000000000000000000000000000000000000000000000000000000000000000000000000000000000000000000000000000801000000000FDFE3C
:4247EE000C000000000000000000000000000000000000000000000000000000000000000000000000000000000000000000000000000000000000000000000000000000FCFE83
:4248300000000000000000000000000000000000000000000000000000000000000000000000000000000000000000000000000000000000000000000000800700000000F8FDCA
:424872000800000000000000000000000000000000000000000000000000000000000000000000000000000000000000000000000000000000000000000000000000008034FE4A
:4248B40000000000000000000000000000000000000000000000000000000000000000000000000000000000000000000000000000000000000000000000800600000000F8FC48
:4248F600000000000000000000000000000000000000000000000000000000000000000000000000000000000000000000000000000000000000000000000000020000001CFE64
:42493800000000000000000000000000000000000000000000000000000000000000000000000000000000000000000000000000000000000000000000000000000000003CFE03
:42497A0000000000000000000000000000000000000000000000000000000000000000000000000000000000000000000000000000000000000000000000800100000000BCFFBF
:4249BC0004000000000000000000000000000000000000000000000000000000000000000000000000000000000000000000000000000000000000000000800000000000EDFF49
:4249FE000C000000000000000000000000000000000000000000000000000000000000000000000000000000000000000000000000000000000000000000001600000000A8FDB0
:424A400000000000000000000000000000000000000000000000000000000000000000000000000000000000000000000000000000000000000000000000800701000000E8FDC7
:424A82000800000000000000000000000000000000000000000000000000000000000000000000000000000000000000000000000000000000000000000000060000008070FCF8
:424AC4000000000000000000000000000000000000000000000000000000000000000000000000000000000000000000000000000000000000000000000000060000000078FC36
:424B06000000000000000000000000000000000000000000000000000000000000000000000000000000000000000000000000000000000000000000000000C00000000012FC9F
:424B4800000000000000000000000000000000000000000000000000000000000000000000000000000000000000000000000000000000000000000000000000000000003CFEF1
:424B8A0000000000000000000000000000000000000000000000000000000000000000000000000000000000000000000000000000000000000000000000800701000000E8FD7C
:424BCC000400000000000000000000000000000000000000000000000000000000000000000000000000000000000000000000000000000000000000000080260000008001FF7D
:424C0E000C00000000000000000000000000000000000000000000000000000000000000000000000000000000000000000000000000000000000000000000100100008074FF54
:424C500000000000000000000000000000000000000000000000000000000000000000000000000000000000000000000000000000000000000000000000800700000000F8FDA6
:424C92000800000000000000000000000000000000000000000000000000000000000000000000000000000000000000000000000000000000000000000000000200008005FF52
:424CD4000000000000000000000000000000000000000000000000000000000000000000000000000000000000000000000000000000000000000000000000160000000068FD23
:424D160000000000000000000000000000000000000000000000000000000000000000000000000000000000000000000000000000000000000000000000800000000000BCFE21
:424D5800000000000000000000000000000000000000000000000000000000000000000000000000000000000000000000000000000000000000000000000000000000003CFEDF
:424D9A0000000000000000000000000000000000000000000000000000000000000000000000000000000000000000000000000000000000000000000000800100000000BCFF9B
:424DDC0004000000000000000000000000000000000000000000000000000000000000000000000000000000000000000000000000000000000000000000800000000000EDFF25
:424E1E000C000000000000000000000000000000000000000000000000000000000000000000000000000000000000000000000000000000000000000000004601000000ACFC57
:424E600000000000000000000000000000000000000000000000000000000000000000000000000000000000000000000000000000000000000000000000800700000000F8FD94
:424EA2000800000000000000000000000000000000000000000000000000000000000000000000000000000000000000000000000000000000000000000000060000008070FCD4
:424EE4000000000000000000000000000000000000000000000000000000000000000000000000000000000000000000000000000000000000000000000000060000000078FC12
:424F2600000000000000000000000000000000000000000000000000000000000000000000000000000000000000000000000000000000000000000000008000000000009EFC2F
:424F6800000000000000000000000000000000000000000000000000000000000000000000000000000000000000000000000000000000000000000000000000000000003CFECD
:424FAA0000000000000000000000000000000000000000000000000000000000000000000000000000000000000000000000000000000000000000000000800100000000BCFF89
:424FEC000400000000000000000000000000000000000000000000000000000000000000000000000000000000000000000000000000000000000000000080000000008065FF1B
:42502E000C00000000000000000000000000000000000000000000000000000000000000000000000000000000000000000000000000000000000000000000160000008020FD81
:4250700000000000000000000000000000000000000000000000000000000000000000000000000000000000000000000000000000000000000000000000800704000000B8FDBE
:4250B2000800000000000000000000000000000000000000000000000000000000000000000000000000000000000000000000000000000000000000000000060000008061FDD0
:4250F4000000000000000000000000000000000000000000000000000000000000000000000000000000000000000000000000000000000000000000000000060000000078FC00
:425136000000000000000000000000000000000000000000000000000000000000000000000000000000000000000000000000000000000000000000000000060200000058FCDB
:42517800000000000000000000000000000000000000000000000000000000000000000000000000000000000000000000000000000000000000000000000000000000003CFEBB
:4251BA0000000000000000000000000000000000000000000000000000000000000000000000000000000000000000000000000000000000000000000000800700000000F8FD37
:4251FC0004000000000000000000000000000000000000000000000000000000000000000000000000000000000000000000000000000000000000000000801002000000DDFE00
:42523E000C000000000000000000000000000000000000000000000000000000000000000000000000000000000000000000000000000000000000000000000000000000FCFE28
:4252800000000000000000000000000000000000000000000000000000000000000000000000000000000000000000000000000000000000000000000000800700000000F8FD70
:4252C2000800000000000000000000000000000000000000000000000000000000000000000000000000000000000000000000000000000000000000000000000000008034FEF0
:425304000000000000000000000000000000000000000000000000000000000000000000000000000000000000000000000000000000000000000000000000060000000078FCED
:42534600000000000000000000000000000000000000000000000000000000000000000000000000000000000000000000000000000000000000000000000000000000001EFC0B
:4253880020000480001000024000080001200004800010000240000800012000040000000000100002400008000120000480001000024000080001200004000010000200B4FC81
:4253CA000000000000000000000000000000000000000000000000000000000000000000000000000000000000000000000000000000000000000000000000040000000078FE27
:42540C0024000480001000024000080001200004800010000240000800012000040000000000100002400008000120000480001000024000080001200004800010000280EDFDBE
:42544E000C00000000000000000000000000000000000000000000000000000000000000000000000000000000000000000000000000000000000000000000000000008074FE1E
:4254900020000480001000024000080001200004800010000240000800012000040000000000100002400008000120000480001000024000080001200004000010000200B4FC78
:4254D2000800000000000000000000000000000000000000000000000000000000000000000000000000000000000000000000000000000000000000000000040000008061FFAC
:425514002000048000100002400008000120000480001000024000080001200004000000000010000240000800012000048000100002400008000120000480001000020034FCF3
:42555600000000000000000000000000000000000000000000000000000000000000000000000000000000000000000000000000000000000000000000000000000000003CFED9
:42559800000000000000000000000000000000000000000000000000000000000000000000000000000000000000000000000000000000000000000000000000000000003CFE97
:4255DA00000000000000000000000000000000000000000000000000000000000000000000000000000000000000000000000000000000000000000000000000000000003CFE55
:42561C00000000000000000000000000000000000000000000000000000000000000000000000000000000000000000000000000000000000000000000000000000000003CFE12
:42565E00000000000000000000000000000000000000000000000000000000000000000000000000000000000000000000000000000000000000000000000000000000003CFED0
:4256A0000000000000000000000000000000000000000000000000000000000000000000000000000000000000000000000000000000000000000000000000000000004078FE12
:4256E200000000000000000000000000000000000000000000000000000000000000000000000000000000000000000000000000000000000000000000000002000000003CFC4C
:42572400000000000000000000000000000000000000000000000000000000000000000000000000000000000000000000000000000000000000000000000000000000003CFE09
:42576600000000000000000000000000000000000000000000000000000000000000000000000000000000000000000000000000000000000000000000000000000000003CFEC7
:4257A800000000000000000000000000000000000000000000000000000000000000000000000000000000000000000000000000000000000000000000000000000000003CFE85
:4257EA00000000000000000000000000000000000000000000000000000000000000000000000000000000000000000000000000000000000000000000000000000000003CFE43
:42582C00000000000000000000000000000000000000000000000000000000000000000000000000000000000000000000000000000000000000000000000000000000003CFE00
:42586E00000000000000000000000000000000000000000000000000000000000000000000000000000000000000000000000000000000000000000000000000010000002CFECD
:4258B000000000000000000000000000000000000000000000000000000000000000000000000000000000000000000000000000000000000000000000000000000000003CFE7C
:4258F200000000000000000000000000000000000000000000000000000000000000000000000000000000000000000000000000000000000000000000000000020000001CFE58
:42593400000100000000000000000000000020000000000000000000000000000000000000000000000000000000000000000000000000000000000000000002000000000CFF03
:42597600000000000000000000000000000000000000000000000000000000000000000000000000000000000000000000000000000000000000000000000002000000003CFCB5
:4259B800000100000000000000000000000000010000000000000000000000000000000000000000000000000000000000000000000000000000000000000000000000003CFF70
:4259FA00000000000000000000000000000000000000000000000000000000000000000000000000000000000000000000000000000000000000000000000000000000003CFE31
:425A3C00000000000000000000000000000000000000000000000000000000000000000000000000000000000000000000000000000000000000000000000000000000003CFEEE
:425A7E00000000000000000000000000000000000000000000000000000000000000000000000000000000000000000000000000000000000000000000000000000000003CFEAC
:425AC000000000000000000000000000000000000000000000000000000000000000000000000000000000000000000000000000000000000000000000000000000000003CFE6A
:425B0200000000000000000000000000000000000000000000000000000000000000000000000000000000000000000000000000000000000000000000000000000000003CFE27
:425B44000000000000000000000000000000000000000000000000000000000000000000000000000000000000000000000000000000000000000000000000040000000078FEA5
:425B8600000000000000000000000000000000000000000000000000000000000000000000000000000000000000000000000000000000000000000000000000000000001EFCC3
:425BC800000000000000000000000000000000000000000000000000000000000000000000000000000000000000000000000000000000000000000000000000000000003CFE61
:425C0A00000000000000000000000000000000000000000000000000000000000000000000000000000000000000000000000000000000000000000000000000000000003CFE1E
:425C4C00000000000000000000000000000000000000000000000000000000000000000000000000000000000000000000000000000000000000000000000000000000003CFEDC
:425C8E00000000000000000000000000000000000000000000000000000000000000000000000000000000000000000000000000000000000000000000000000000000003CFE9A
:425CD000000000000000000000000000000000000000000000000000000000000000000000000000000000000000000000000000000000000000000000000000000000003CFE58
:425D1200000000000000000000000000000000000000000000000000000000000000000000000000000000000000000000000000000000000000000000000000000000003CFE15
:425D5400000000000000000000000000000000000000000000000000000000000000000000000000000000000000000000000000000000000000000000000000000000003CFED3
:425D960000000000000000000000000000000000000000000000000000000000000000000000000000000000000000000000000000000000000000000000800100000000BCFF8F
:425DD800000000000000000000000000000000000000000000000000000000000000000000000000000000000000000000000000000000000000000000000001000000003CFF4D
:425E1A00000000000000000000000000000000000000000000000000000000000000000000000000000000000000000000000000000000000000000000000000000000003CFE0C
:425E5C000000000000000000000000000000000000000000000000000000000000000000000000000000000000000000000000000000000000000000000000000000004078FE4E
:425E9E00000000000000000000000000000000000000000000000000000000000000000000000000008200000000000000008000000000000000000000000000000000001CFCA8
:425EE0000000000000000000000000000000000000000000000000000000000000000000000000000000000000000000000000000000000000000000000000000000004078FECA
:425F220000000000000000000000000000000000000000000000000000000000000000000000000000880000000000000000000200000000000000000000000201000000A4FE0E
:425F64000000000000000000000000000000000000000000000000000000000000000000000000000000000010040000000000000000000000000002000000000200000068FC7F
:425FA6000000000000000000000000000000000000000000000000000000000000000000000000000000000020080000000000000000000000000001000000000000000084FF0D
:425FE800000000000000000000000000000000000000000000000000000000000000000000000000000000000000000000000000000000000000000000000000000000003CFE3D
:42602A00000000000000000000000000000000000000000000000000000000000000000000000000000000000000000000000000000000000000000000000000000000003CFEFA
:42606C00000000000000000000000000000000000000000000000000000000000000000000000000000000000000000000000000000000000000000000000000000000003CFEB8
:4260AE00000000000000000000000000000000000000000000000000000000000000000000000000000000000000000000000000000000000000000000000000000000003CFE76
:4260F000000000000000000000000000000000000000000000000000000000000000000000000000000000000000000000000000000000000000000000000000000000003CFE34
:42613200000000000000000000000000000000000000000000000000000000000000000000000000000000000000000000000000000000000000000000000000000000003CFEF1
:42617400000000000000000000000000000000000000000000000000000000000000000000000000000000000000000000000000000000000000000000000000000000003CFEAF
:4261B600000000000000000000000000000000000000000000000000000000000000000000000000000000000000000000000000000000000000000000000000000000002DFF7B
:4261F800000000000000000000000000000000000000000000000000000000000000000000000000000000000000000000000000000000000000000000000000000000003CFE2B
:42623A00000000000000000000000000000000000000000000000000000000000000000000000000000000000000000000000000000000000000000000000000000000003CFEE8
:42627C00000000000000000000000000000000000000000000000000000000000000000000000000000000000000000000000000000000000000000000000000010000002CFEB5
:4262BE00000000000000000000000000000000000000000000000000000000000000000000000000000000000000000000000000000000000000000000000000000000003CFE64
:42630000000000000000000000000000000000000000000000000000000000000000000000000000000000000000000000000000000000000000000000000000000000003CFE21
:42634200000000000000000000000000000000000000000000000000000000000000000000000000000000000000000000000000000000000000000000000000000000003CFEDF
:42638400000000000000000000000000000000000000000000000000000000000000000000000000000000000000000000000000000000000000000000000000000000003CFE9D
:4263C600000000000000000000000000000000000000000000000000000000000000000000000000000000000000000000000000000000000000000000000000000000003CFE5B
:42640800000000000000000000000000000000000000000000000000000000000000000000000000000000000000000000000000000000000000000000000000000000003CFE18
:42644A00000000000000000000000000000000000000000000000000000000000000000000000000000000000000000000000000000000000000000000000000000000003CFED6
:42648C00000000000000000000000000000000000000000000000000000000000000000000000000000000000000000000000000000000000000000000000000000000003CFE94
:4264CE00000000000000000000000000000000000000000000000000000000000000000000000000000000000000000000000000000000000000000000000000000000003CFE52
:42651000000000000000000000000000000000000000000000000000000000000000000000000000000000000000000000000000000000000000000000000000000000003CFE0F
:4265520000040000000000000000000000000000000000001A0000000000000000000000000000000000000000000000000000000000000000000000000000000000000082FF68
:4265940000800000000000000000000000000000000000000000000000000000000000000000000000000000000000000000000000000000000000000000000000000000BCFE8B
:4265D600E0010000000000000000000000000000000000001E000000000000000000000000000000000000000000000000000000000000000000000000000000000000003CFE4A
:42661800A8010000000000000000000000000000000000000204000000000000000000000000000000000000000000000000000000000000000000000000000000000080FDFE16
:42665A00801100000000000000000000000000000000000000050000000000000000000000000000000000000000000000000000000000000000000000000000000000806CFF7D
:42669C00E0410000000000000000000000000000000000001E000000000000000000000000000000000000000000000000000000000000000000000000000000000000007CFE03
:4266DE0004000000000000000000000000000000000000000000000000000000000000000000000000000000000000000000000000000000000000000000000000000080E5FF12
:426720002050000000000000000000000000000000000000400400000000000000000000000000000000000000000000000000000000000000000000000000000000000028FC5F
:426762002048000000000000000000000000000000000000020000000000000000000000000000000000000000000000000000000000000000000000000000000000000074FE19
:4267A400000000000000000000000000000000000000000000000000000000000000000000000000000000000000000000000000000000000000000000000000000000003CFE79
:4267E600E0400000000000000000000000000000000000001E000000000000000000000000000000000000000000000000000000000000000000000000000000000000006CFFC8
:4268280024000000000000000000000000000000000000001A00000000000000000000000000000000000000000000000000000000000000000000000000000000000000F5FEFD
:42686A008C050000000000000000000000000000000000001805000000000000000000000000000000000000000000000000000000000000000000000000000000000000A8FE98
:4268AC00E0410000000000000000000000000000000000001E000000000000000000000000000000000000000000000000000000000000000000000000000000000000007CFEF1
:4268EE0088410000000000000000000000000000000000000000000000000000000000000000000000000000000000000000000000000000000000000000000000000080ECFF34
:4269300080040000000000000000000000000000000000004004000000000000000000000000000000000000000000000000000000000000000000000000000000000000F4FE6B
:4269720080050000000000000000000000000000000000008A0000000000000000000000000000000000000000000000000000000000000000000000000000000000000002FFD3
:4269B4008081000000000000000000000000000000000000100400000000000000000000000000000000000000000000000000000000000000000000000000000000000074FE1A
:4269F600E0010000000000000000000000000000000000000604000000000000000000000000000000000000000000000000000000000000000000000000000000000000E4FF91
:426A3800A8010000000000000000000000000000000000004200000000000000000000000000000000000000000000000000000000000000000000000000000000000080B9FEFA
:426A7A00000800000000000000000000000000000000000088040000000000000000000000000000000000000000000000000000000000000000000000000000000000807CFE4C
:426ABC0060400000000000000000000000000000000000000E00000000000000000000000000000000000000000000000000000000000000000000000000000000000000F4FEF8
:426AFE0004000000000000000000000000000000000000000004000000000000000000000000000000000000000000000000000000000000000000000000000000000080A5FF2A
:426B40002000000000000000000000000000000000000000800000000000000000000000000000000000000000000000000000000000000000000000000000000000000034FC43
:426B8200A0010000000000000000000000000000000000001A000000000000000000000000000000000000000000000000000000000000000000000000000000000000001EFCFC
:426BC40000000000000000000000000000000000000000001800000000000000000000000000000000000000000000000000000000000000000000000000000000000000A4FFD4
:426C0600E0410000000000000000000000000000000000001E000000000000000000000000000000000000000000000000000000000000000000000000000000000000007CFE93
:426C480028100000000000000000000000000000000000001A00000000000000000000000000000000000000000000000000000000000000000000000000000000000080ADFE8D
:426C8A0000500000000000000000000000000000000000008004000000000000000000000000000000000000000000000000000000000000000000000000000000000080ACFECA
:426CCC00E001000000000000000000000000000000000000060000000000000000000000000000000000000000000000000000000000000000000000000000000000000086FD1C
:426D0E0084410000000000000000000000000000000000000000000000000000000000000000000000000000000000000000000000000000000000000000000000000000B5FECB
:426D50000004000000000000000000000000000000000000000000000000000000000000000000000000000000000000000000000000000000000000000000000000000038FEC7
:426D920030000000000000000000000000000000000000001A0000000000000000000000000000000000000000000000000000000000000000000000000000000000000086FCF3
:426DD400000000000000000000000000000000000000000000000000000000000000000000000000000000000000000000000000000000000000000000000000000000003CFE43
:426E1600E0010000000000000000000000000000000000000604000000000000000000000000000000000000000000000000000000000000000000000000000000000000E4FF6C
:426E5800A4010000000000000000000000000000000000005A00000000000000000000000000000000000000000000000000000000000000000000000000000000000080E1FF99
:426E9A00845100000000000000000000000000000000000000040000000000000000000000000000000000000000000000000000000000000000000000000000000000807CFFE2
:426EDC00E0010000000000000000000000000000000000000600000000000000000000000000000000000000000000000000000000000000000000000000000000000000A4FFEA
:426F1E000C40000000000000000000000000000000000000000400000000000000000000000000000000000000000000000000000000000000000000000000000000008065FFFD
:426F60000004000000000000000000000000000000000000000100000000000000000000000000000000000000000000000000000000000000000000000000000000000028FEC4
:426FA200A0010000000000000000000000000000000000000200000000000000000000000000000000000000000000000000000000000000000000000000000000000000A4FF67
:426FE40080010000000000000000000000000000000000000000000000000000000000000000000000000000000000000000000000000000000000000000000000000000A4FF47
:42702600E0010000000000000000000000000000000000000000000000000000000000000000000000000000000000000000000000000000000000000000000000000000E0FD6A
:42706800A40100000000000000000000000000000000000000050000000000000000000000000000000000000000000000000000000000000000000000000000000000802DFC93
:4270AA000C5000000000000000000000000000000000000080040000000000000000000000000000000000000000000000000000000000000000000000000000000000806CFEDA
:4270EC00600000000000000000000000000000000000000006000000000000000000000000000000000000000000000000000000000000000000000000000000000000003CFEC2
:42712E000800000000000000000000000000000000000000000400000000000000000000000000000000000000000000000000000000000000000000000000000000008065FF2F
:4271700000000000000000000000000000000000000000005800000000000000000000000000000000000000000000000000000000000000000000000000000000000000A0FFE6
:4271B200200000000000000000000000000000000000000002000000000000000000000000000000000000000000000000000000000000000000000000000000000000003CFE3F
:4271F400000000000000000000000000000000000000000000000000000000000000000000000000000000000000000000000000000000000000000000000000000000003CFE1F
:4272360080010000000000000000000000000000000000000000000000000000000000000000000000000000000000000000000000000000000000000000000000000000A4FFF2
:4272780084010000000000000000000000000000000000000004000000000000000000000000000000000000000000000000000000000000000000000000000000000000B5FE98
:4272BA008C11000000000000000000000000000000000000000500000000000000000000000000000000000000000000000000000000000000000000000000000000000024FFCD
:4272FC00E0410000000000000000000000000000000000000600000000000000000000000000000000000000000000000000000000000000000000000000000000000000E4FF46
:42733E0008000000000000000000000000000000000000001800000000000000000000000000000000000000000000000000000000000000000000000000000000000080ACFFC2
:42738000004400000000000000000000000000000000000040040000000000000000000000000000000000000000000000000000000000000000000000000000000000003CFE09
:4273C200000100000000000000000000000000000000000000000000000000000000000000000000000000000000000000000000000000000000000000000000000000000EFD7D
:427404000000048000100002400008000120000480001000024000080001200004000000000010000240000800012000048000100002400008000120000480001000020034FE02
:42744600000000000000000000000000000000000000000000000000000000000000000000000000000000000000000000000000000000000000000000000000000000003CFECA
:42748800280004800010000240000800012000048000100002400008000120000400000000001000024000080001200004800010000240000800012000048000100002802DFDDE
:4274CA0000010000000000000000000000000000000000000000000000000000000000000000000000000000000000000000000000000000000000000000000000000080A4FF5C
:42750C000000048000100002400008000120000480001000004000080001200004000000000010000240000800012000048000100002400008000120000480001000020034FCFD
:42754E0004000000000000000000000000000000000000001000000000000000000000000000000000000000000000000000000000000000000000000000000000000080F5FE74
:427590002000048000100002400008000120000480001000024000080001200004000000000010000240000800012000048000100002400008000120000480001000020034FC57
:4275D200000000000000000000000000000000000000000000000000000000000000000000000000000000000000000000000000000000000000000000000000000000003CFE3D
:42761400000000000000000000000000000000000000000000000000000000000000000000000000000000000000000000000000000000000000000000000000000000003CFEFA
:42765600000000000000000000000000000000000000000000000000000000000000000000000000000000000000000000000000000000000000000000000000000000003CFEB8
:42769800000000000000000000000000000000000000000000000000000000000000000000000000000000000000000000000000000000000000000000000000000000003CFE76
:4276DA00000000000000000000000000000000000000000000000000000000000000000000000000000000000000000000000000000000000000000000000000000000003CFE34
:42771C00000000000000000000000000000000000000000000000000000000000000000000000000000000000000000000000000000000000000000000000000000000003CFEF1
:42775E00000000000000000000000000000000000000000000000000000000000000000000000000000000000000000000000000000000000000000000000000000000003CFEAF
:4277A000000000000000000000000000000000000000000000000000000000000000000000000000000000000000000000000000000000000000000000000000000000003CFE6D
:4277E200000000000000000000000000000000000000000000000000000000000000000000000000000000000000000000000000000000000000000000000000000000C0F0FEB7
:42782400000000000000000000000000000000000000000000000000000000000000000000000000000000000000000000000000000000000000000000000000000000003CFEE8
:42786600000000000000000000000000000000000000000000000000000000000000000000000000000000000000000000000000000000000000000000000000000000003CFEA6
:4278A800000000000000000000000000000000000000000000000000000000000000000000000000000000000000000000000000000000000000000000000000000000001EFC84
:4278EA00000000000000000000000000000000000000000000000000000000000000000000000000100000000000010000000000000000000000000000000000000000002CFF20
:42792C00000000000000000000000000000000000000000000000000000000000000000000000000000000000000000000000000000000000000000000000000000000003CFEDF
:42796E00000000000000000000000000000000000000000000000000000000000000000000000000040000000000040000000000000000000000000000000000000000003CFE95
:4279B000000000000000000000000000000000000000000000000000000000000000000000000000000000000000000000000000000000000000040000000000000000007CFE17
:4279F20000000000000000000000000000000000000000000000000000000000000000000000000000000000000000000000000000000000000008000000000000000000BCFE91
:427A3400000000000000000000000000000000000000000000000000000000000000000000000000000000000000000000000000000000000000000000000000000000003CFED6
:427A7600000000000000000000000000000000000000000000000000000000000000000000000000000000000000000000000000000000000000000000000000000000003CFE94
:427AB800000000000000000000000000000000000000000000000000000000000000000000000000000000000000000000000000000000000000000000000000000000003CFE52
:427AFA00000000000000000000000000000000000000000000000000000000000000000000000000000000000000000000000000000000000000000000000000000000003CFE10
:427B3C00000000000000000000000000000000000000000000000000000000000000000000000000000000000000000000000000000000000000000000000000000000003CFECD
:427B7E00000000000000000000000000000000000000000000000000000000000000000000000000000000000000000000000000000000000000000000000000000000003CFE8B
:427BC000000000000000000000000000000000000000000000000000000000000000000000000000000000000000000000000000000000000000000000000000000000003CFE49
:427C0200000000000000000000000000000000000000000000000000000000000000000000000000000000000000000000000000000000000000000000000000000000003CFE06
:427C4400000000000000000000000000000000000000000000000000000000000000000000000000000000000000000000000000000000000000000000000000000000001EFCE4
:427C8600000000000000000000000000000000000000000000000000000000000000000000000000000000000000000000000000000000000000000000000000000000003CFE82
:427CC800000000000000000000000000000000000000000000000000000000000000000000000000000000000000000000000000000000000000000000000000000000003CFE40
:427D0A00000000000000000000000000000000000000000000000000000000000000000000000000000000000000000000000000000000000000000000000000000000003CFEFD
:427D4C00000000000000000000000000000000000000000000000000000000000000000000000000000000000000000000000000000000000000000000000000000000003CFEBB
:427D8E00000000000000000000000000000000000000000000000000000000000000000000000000000000000000000000000000000000000000000000000000000000003CFE79
:427DD000000000000000000000000000000000000000000000000000000000000000000000000000000000000000000000000000000000000000000000000000000000003CFE37
:427E1200000000000000000000000000000000000000000000000000000000000000000000000000000000000000000000000000000000000000000000000000000000003CFEF4
:427E5400000000000000000000000000000000000000000000000000000000000000000000000000000000000000000000000000000000000000000000000000000000003CFEB2
:427E9600000000000000000000000000000000000000000000000000000000000000000000000000000000000000000000000000000000000000000000000000000000003CFE70
:427ED800000000000000000000000000000000000000000000000000000000000000000000000000000000000000000000000000000000000000000000000000000000003CFE2E
:427F1A000000000000000000000000000000000000000000000000000000000000000000000000000000000000000000000000000000000000000000000000000010004068FE6F
:427F5C00000000000000000000000000000000000000000000000000000000000000000000000000000000000000000000000000000000000000000000000000000000001EFCC9
:427F9E000000000000000000000000000000006000000000000000000000000000000000000000000000000000000000000000000000000000000000000000000040000038FCCD
:427FE00040000000000000000000000000000000000000000800000000000000000000000000000000000000000000000000000000000000000000000000000000000000F0FE29
:4280220000000000000000000000000000000000000000000800000000000000000000000000000000000000000000000000000000000000000000000000000000000000B4FE62
:42806400000000000000000000000000000000000000000000000000000000000000000000000000000000000000000000000000000000000000000000000000000000003CFEA0
:4280A600000000000000000000000000000000000000000000000000000000000000000000000000000000000000000000000000000000000000000000000000000000003CFE5E
:4280E800000000000000000000000000000000000000000000000000000000000000000000000000000000000000000000000000000000000000000000000000000000003CFE1C
:42812A00000000000000000000000000000000000000000000000000000000000000000000000000000000000000000000000000000000000000000000000000000000003CFED9
:42816C00000000000000000000000000000000000000000000000000000000000000000000000000000000000000000000000000000000000000000000000000000000003CFE97
:4281AE00000000000000000000000000000000000000000000000000000000000000000000000000000000000000000000000000000000000000000000000000000000003CFE55
:4281F000000000000000000000000000000000000000000000000000000000000000000000000000000000000000000000000000000000000000000000000000000000003CFE13
:42823200000000000000000000000000000000000000000000000000000000000000000000000000000000000000000000000000000000000000000000000000000000003CFED0
:42827400000000000000000000000000000000000000000000000000000000000000000000000000000000000000000000000000000000000000000000000000000000003CFE8E
:4282B600000000000000000000000000000000000000000000000000000000000000000000000000000000000000000000000000000000000000000000000000000000003CFE4C
:4282F800000100000000000000000000000000000000000000000000000000000000000000000000000000000000000000000000000000000000000000000000000000002CFF18
:42833A00000000000000000000000000000000000000000000000000000000000000000000000000000000000000000000000000000000000000000000000000000000001EFCE7
:42837C00000000000000000000000000000000000000000000000000000000000000000000000000000000000000000000000000000000000000000000000000000000003CFE85
:4283BE0000000000000000000000000000000000000000000000000000000000000000000000000000000000000004000000000000000000000000040000000000840000FCFEF7
:42840000000000000000000000000000000000000000000000000000000000000000000000000000000000000000000000000000000000000000000000000000000000003CFE00
:42844200000000000000000000000000000000000000000000000000000000000000000000000000000000000003000000000000000000000000030000000000F0200000E0FE04
:42848400000000000000000000000000000000000000000000000000000000000000000000000000000000000001000000000000000000000000010000000000D0000000E0FE06
:4284C60000000000000000000000000000000000000000000000000000000000000000000000000000000000002C0200000000000000000000008C000000000000040000BCFCFE
:4285080000000000000000000000000000000000000000000000000000000000000000000000000000000000000F0000000000000000000000000F0200000000F0400000ACFC39
:42854A0000000000000000000000000000000000000000000000000000000000000000000000000000000000000C0000000000000000000000000C00000000000040000070FE29
:42858C0000000000000000000000000000000000000000000000000000000000000000000000000000000000000D0000000000000000000000000C0000000000C0040000F8FFD9
:4285CE0000000000000000000000000000000000000000000000000000000000000000000000000000000000000C1000000000000000000000008C0400000000C04800001AFDA0
:42861000000000000000000000000000000000000000000000000000000000000000000000000000000000000000000000000000000000000000000000000000000000003CFEEE
:4286520000000000000000000000000000000000000000000000000000000000000000000000000000000000000F0400000000000000000000000F0400000000F0400000C8FECA
:428694000800000000000000000000000000000000000000000000000000000000000000000000000000000000210000000000000000000000002100000000001002008035FD96
:4286D60000000000000000000000000000000000000000000000000000000000000000000000000000000000000000000000000000000000000000000000000000000080B4FE30
:4287180000000000000000000000000000000000000000000000000000000000000000000000000000000000000F0000000000000000000000000F0000000000F0000000EEFC27
:42875A00040000000000000000000000000000000000000000000000000000000000000000000000000000000000000000000000000000000000000000000000000000006DFF6D
:42879C0000000000000000000000000000000000000000000000000000000000000000000000000000000000000C0000000000000000000000000D0000000000D0000000ECFFC7
:4287DE000000000000000000000000000000000000000000000000000000000000000000000000000000000000000400000000000000000000008C0400000000C0480000B4FE0B
:42882000000000000000000000000000000000000000000000000000000000000000000000000000000000000000000000000000000000000000000000000000000000003CFEDC
:428862000000000000000000000000000000000000000000000000000000000000000000000000000000000000030000000000000000000000000F0800000000F000000008FEC4
:4288A40004000000000000000000000000000000000000000000000000000000000000000000000000000000000100000000000000000000000081000000000010100000E5FF08
:4288E6000C000000000000000000000000000000000000000000000000000000000000000000000000000000008C0200000000000000000000000000000000000000000018FEA0
:4289280000000000000000000000000000000000000000000000000000000000000000000000000000000000000F0000000000000000000000000F0000000000F0000000CCFE35
:42896A0008000000000000000000000000000000000000000000000000000000000000000000000000000000000C00000000000000000000000000000000000000000080F8FE41
:4289AC0000000000000000000000000000000000000000000000000000000000000000000000000000000000000D0000000000000000000000000D0000000000D0000000ECFEB5
:4289EE00802100000000000000030200000000000000000000000000008C1000000000000000000000000000000004000000000000000000000080010000000000000000F2FF8F
:428A3000000000000000000000000000000000000000000000000000000000000000000000000000000000000000000000000000000000000000000000000000004000007CFE4A
:428A7200E001000000000000C0030000000000000000000000000000000F080000000000000000000000000000030000000000000000000000000F020000000030000000B8FC0F
:428AB4002800010000000000405000000000000000000000000000000081000000000000000000000000000000010000000000000000000000008D000000000010000080ADFC7F
:428AF60000000000000000000000000000000000000000000000000000000000000000000000000000000000008C000000000000000000000000400000000000C0080080F0FE3C
:428B3800E001000000000000C0030000000000000000000000000000000F0000000000000000000000000000000F0200000000000000000000000F0400000000F020000014FE02
:428B7A0004000000000000000000000000000000000000000000000000000000000000000000000000000000000C000000000000000000000000000400000000C0000080E1FF85
:428BBC00800100000000000000030000000000000000000000000000000C0000000000000000000000000000000D0000000000000000000000002C0000000000C000000058FC9A
:428BFE000000000000000000000000000C811102000000000000000000000000000000000000000000000000000C1000000000000000000000000C04000000000000000076FCF7
:428C4000000000000000000000000000000000000000000000000000000000000000000000000000000000000000000000000000000000000000000000000000004000007CFE38
:428C82000000000000000000000000000FE00100000000000000000000000000000000000000000000000000000F0400000000000000000000000F00000000003000000050FF1F
:428CC4000400000000000000000000000124000100000000000000000000000000000000000000000000000000010000000000000000000000004110000000001000008085FFDE
:428D06000C0000000000000000000000000000000000000000000000000000000000000000000000000000000000000000000000000000000000000000000000C002008098FC49
:428D48000000000000000000000000000FE00100000000000000000000000000000000000000000000000000000F0000000000000000000000000F0000000000F0200000DEFDF0
:428D8A00080000000000000000000000000000000000000000000000000000000000000000000000000000000000000000000000000000000000000000000000C000000061FF7F
:428DCC000000000000000000000000000C800100000000000000000000000000000000000000000000000000000C0000000000000000000000000C0000000000C0000000BCFF45
:428E0E0000000000000000000000000000000000000000000000000000000000000000000000000000000000000C1000000000000000000000000004000000000084000052FD2F
:428E5000000000000000000000000000000000000000000000000000000000000000000000000000000000000000000000000000000000000000000000000000000000003CFEA6
:428E920000000000000000000000000000000000000000000000000000000000000000000000000000000000000F080000000000000000000000030000000000F0200000ACFECA
:428ED400080000000000000000000000000000000000000000000000000000000000000000000000000000000041000000000000000000000000010000000000D0040080F9FFC6
:428F16000000000000000000000000000000000000000000000000000000000000000000000000000000000000000000000000000000000000002C00000000000004008070FCFD
:428F580000000000000000000000000000000000000000000000000000000000000000000000000000000000000F0000000000000000000000000F0200000000F04000008EFEFB
:428F9A000400000000000000000000000000000000000000000000000000000000000000000000000000000000000000000000000000000000000C000000000000400000EDFF59
:428FDC0000000000000000000000000000000000000000000000000000000000000000000000000000000000000C0000000000000000000000000C0000000000C0020000DCFCA1
:42901E0000000000000000000000000000000000000000000000230400000000000000000000000000000000000C1000000000000000000000000C0400000000C00000008EFE71
:42906000000000000000000000000000000000000000000000000000000000000000000000000000000000000000000000000000000000000000000000000000004000007CFE14
:4290A200000000000000000000000000000000000000000000C0030000000000000000000000000000000000000F0000000000000000000000000F0800000000F0800000B8FD7E
:4290E4000400000000000000000000000000000000000000004000010000000000000000000000000000000000811000000000000000000000008100000000001004008035FF2B
:429126000C00000000000000000000000000000000000000000000000000000000000000000000000000000000000000000000000000000000000000000000000000008074FE09
:42916800000000000000000000000000000000000000000000C0030000000000000000000000000000000000000F0000000000000000000000000F0000000000F000000012FFE3
:4291AA0008000000000000000000000000000000000000000000000000000000000000000000000000000000000000000000000000000000000000000000000000000000ADFFCF
:4291EC0000000000000000000000000000000000000000000000030000000000000000000000000000000000000C0000000000000000000000000C0000000000C0000000CCFD9D
:42922E008021000000000000000302000C8111020000000000002304000000000000000000000000000000000000040000000000000000000000800100000000C0000000B4FE9A
:42927000000000000000000000000000000000000000000000000000000000000000000000000000000000000000000000000000000000000000000000000000004000007CFE02
:4292B200E081000000000000C00301000FE881000000000000C003010000000000000000000000000000000000030000000000000000000000000F0200000000F0000000BCFD5C
:4292F4002410000000000000400000008120100000000000004000000000000000000000000000000000000000010000000000000000000000000D00000000001010000055FC54
:429336000C000000000000000000000000000000000000000000000000000000000000000000000000000000004C0200000000000000000000004000000000000000000050FE0D
:42937800E001000000000000C00300000FE001000000000000C0030000000000000000000000000000000000000F0000000000000000000000000F0400000000F0000000C4FF87
:4293BA0008000000000000000000000000000000000000000000000000000000000000000000000000000000000C00000000000000000000000000040000000000000080FCFEDF
:4293FC008001000000000000000300000C800100000000000000030000000000000000000000000000000000000D0000000000000000000000008C0000000000C0000000ACFC1A
:42943E000000000000000000000000000000000000000000000000000000000000000000000000000000000000080000000000000000000000000000000000000000000096FC52
:429480002000048000100002400008000120000480001000024000080001200004000000000010000240000800002000048000100002400008000020000480000000020024FC6A
:4294C2000000000000000000000000000000000000000000000000000000000000000000000000000000000000000000000000000000000000000800000000008000000034FEAE
:42950400280004800010000240000800012000048000100002400008000120000400000000001000024000080001200004800010000240000800012000048000100002802DFD41
:42954600000000000000000000000000000000000000000000000000000000000000000000000000000000000008000000000000000000000000000000000000000000803CFE21
:429588000000048000100002000008000000000480001000020000080000200004000000000010000240000800002000048000100002400008000020000480000000020066FDE0
:4295CA0004010000000000000002000008000100000000000000020000080000000000000000000000000000000000000000000000000000000008000000000080000000FDFDC3
:42960C002000048000100002400008000120000480001000024000080001200004000000000010000240000800012000048000100002400008000120000480001000020034FCBA
:42964E000000000000000000000000000000000000000000000000000000000000000000000000000000000000040000000000000000000000000000000000000000000078FE60
:42969000000000000000000000000000000000000000000000000000000000000000000000000000000000000000000000000000000000000000040000000000000000007CFE1A
:4296D200000000000000000000000000000000000000000000000000000000000000000000000000000000000000000000000000000000000000000000000000000000003CFE1C
:429714000000000000000000000000000000000000000000000000000000000000000000000000000000000000000000000000000000000000000000000000000000004078FE5D
:42975600000000000000000000000000000000000000000000000000000000000000000000000000000000000000000000000000000000000000000000000000100000003CFF86
:4297980000000000000000000000000000000001000000000000000200000800000000000000000000000000000000000000000000000000000000010000000000000000B4FDD2
:4297DA00000000000000000000000000000000000000000000000000000000000000000000000000000000000000000000000000000000000000000000000000000000003CFE13
:42981C00000000000000000000000000000000000000000000000000000000000000000000000000000000000000000000000000000000000000000000000000000000003CFED0
:42985E00000000000000000000000000000000000000000000000000000000000000000000000000000000000000000000000000000000000000000000000000000000001EFCAE
:4298A000000000000000000000000000000000000000000000000000000000000000000000000000000000000000000000000000000000000000000000000000000000003CFE4C
:4298E2000000000000000000000000000000000000000000000000000000000000000000000000000000000000200000000000000000000000000008000000002000000014FEEA
:429924000000000000000000000000000000000000000000000000000000000000000000000000000000000000000000000000000000000000000000000000000000004078FE4B
:42996600000000000000000000000000000000000000000000000000000000000000000000000040000000000004000000000000000000000000000000000000000000007CFE01
:4299A8000000000000000000000000000008000000000000000000000000000000000000000000000000000000000000000000000000000000000000000000000000000034FE43
:4299EA000000100000000000000000000008000000000000000000000000000000000000000000400000000000420100000000000000000000004001000000000000500074FD9E
:429A2C000000A00000000032000200000000000004848000100000C8000000000000000000000000000000000002000000008000000000000000020000000000000068007CFFDD
:429A6E0000000000000000000000000000000000000000000000000000000000000000000000000000000000000000000000000000000000000000000000000000000800B4FEFC
:429AB0000000200000000010000200000000000020048400100000400000000000000000000000000000000000000000000080000000000000000000000000000000000014FDB9
:429AF200000000000000000000000000000000000000000000000000000000000000000000000000000000000000000000000000000000000000040000000000000000007CFEB4
:429B3400000000000000000000000000000000000000000000000000000000000000000000000000000000000002000000000000000000000000000000000000000000003CFCB5
:429B7600000000000000000000000000000000000000000000000000000000000000000000000000000000000000000000000000000000000000000000000000000000003CFE73
:429BB800000000000000000000000000000000000000000000000000000000000000000000000000000000000000000000000000000000000000000000000000000000003CFE31
:429BFA00000000000000000000000000000000000000000000000000000000000000000000000000000000000000000000000000000000000000000000000000000200001CFC0F
:429C3C00000000000000000000000000000000000000000000000000000000000000000000000000000000000000100000000000000000000000000000000000000000003CFF9B
:429C7E0000000000000000000000000000000000000000000000000000000000000000000000000000000000000000000000000000000000000000000000000040000080F0FEF6
:429CC000000000000000000000000000000000000000000000000000000000000000000000000000000000000000000000000000000000000000000000000000000000003CFE28
:429D0200000000000000000000000000000000000000000000000000000000000000000000000000000000000000000000000000000000000000000000000000000000003CFEE5
:429D4400000000000000000000000000000000000000000000000000000000000000000000000000000000000000000000000000000000000000000000000000000000003CFEA3
:429D8600000000000000000000000000000000000000000000000000000000000000000000000000000000000000000000000000000000000000000000000000000000003CFE61
:429DC8000000000000000000400000000000000000000000000000000000000000000000000000000000000000000000000000000000000000000000000000000000000038FEE3
:429E0A0000800000000000000000000010008000000000000000040000000000000000000000000000000000000000000000000000000000000000000000000000000000B0FF53
:429E4C0080000000000000008000000000800000000000000080000000000000000000000000000000000000000000000000000000000000000000000000000000000000B4FE22
:429E8E000000000000000000000000000000000000000000000000000000000000000000000000000000000000020800000000000000000000000B00000000008000000084FC7D
:429ED000000000000000000000000000000000000000000000000000000000000000000000000000000000000000000000000000000000000000020000000000201100001CFD04
:429F120000000000000000000008000000000000000000000000000000000000000000000000000000000000000000000000000000000000000000000000000000000000BCFE4B
:429F5400200000000000000000000000010000000000000000000000000000000000000000000000000000000000000000000000000000000000000000000000000000002CFC82
:429F9600000000000000000000000000000000080000000000000000000000000000000000000000000200000000000000008000000000000000000000000000020000405AFE65
:429FD800000000000000000000000000000000000000000000000000000000000000000000000000000000000000000000000000000000000000000000000000000000003CFE0D
:42A01A0000000000000000000000000A8001000800000000000001000000000000000000000000000008000000000000000000020000000000000000000000000214000080FED2
:42A05C002000000000000000400000020240004800000000220000000000000000000000000000000000000010020000000080000000000000000404000000000120000058FCA5
:42A09E00000000000000000000000000000000000000000000000000000000000000000000000000000000002000000000000000000000000000040000000000022000005CFEE0
:42A0E00000000000000000000000000000000000000000000000000000000000000000000000000000000000000000000000800000000000000000000000000000000000BCFE04
:42A12200100000000000000000000000000000000000000000000000000000000000000000000000000000000000000000000000000000000000000000000000000000001EFDD0
:42A16400000000000000000000000000000000000000000000000000000000000000000000000000000000000000000000000000000000000000000000000000000000003CFE7F
:42A1A600000000000000000000000000000000000000000000000000000000000000000000000000000000000000000000000000000000000000000000000000000000003CFE3D
:42A1E80004000000000000000000000000000000000000000000000000000000000000000000000000000000000000000000000000000000000000000000000000000080F4FEBF
:42A22A00040000000000000000000000000000000000000000000000000000000000000000000000000000000000000000000000000000000000000000000000000000400BFDA6
:42A26C00000000000000000000000000000000000000000000000000000000000000000000000000000000000000000000000000000000000000000000000000000000003CFE76
:42A2AE00000000000000000000000000000000000000000000000000000000000000000000000000000000000000000000000000000000000000000000000000000000001EFC54
:42A2F000000000000000000000000000000000000000000000000000000000000000000000000000000000000000000000000000000000000000000000000000000000003CFEF2
:42A33200000000000000000000000000000000000000000000000000000000000000000000000000000000000000000000000000000000000000000000000000000000003CFEAF
:42A374000000000000000000000000000001000000000000000000000000010000000000000000000000000000000000000000000000000000000000000000000000004079FFED
:42A3B600000000000000000000000000000000000000000000000000000000000000000000000000000000000000000000000000000000000000000000000000000000003CFE2B
:42A3F800000000000000000000000000000000000000000000000000000000000000000000000000000000000000000000000000000000000000000000000000000000003CFEE9
:42A43A00000000000000000000000000000000000000000000000000000000000000000000000000000000001100000000000000000000000000000000000000000000003CFF94
:42A47C00000000000000000000000000000000000000000000000000000000000000000000000000000000000000000000000000000000000000000000000000000000003CFE64
:42A4BE0000000000000000000000000000000000000000000000000000000000000000000000000000000078000000000000000000000000000000000000000000000000F8FDEF
:42A5000000000000000000000000000000000000000000000000000000000000000000000000000000000068140000000000000000000000000000000000000000000000ECFCB5
:42A54200000000000000000000000000000000000000000000000000000000000000000000000000000000008200000000000000000000000000000000000000000000009CFCBD
:42A5840000000000000000000000000000000000000000000000000000000000000000000000000000000078000000000000000000000000000000000000000000000000F8FD28
:42A5C600000000000000000000000000000000000000000000000000000000000000000000000000000000000000000000000000000000000000000000000000000000003CFE19
:42A608000000000000000000000000000000000000000000000000000000000000000000000000000000006042000000000000000000000000000000000000000000000018FE58
:42A64A0000000000000000000000000000000000000000000000000000000000000000000000000000000060800000000000000000000000000000000000000000000000DAFE16
:42A68C00000000000000000000000000000000000000000000000000000000000000000000000000000000000000000000000000000000000000000000000000000000003CFE52
:42A6CE0000000000000000000000000000000000000000000000000000000000000000000000000000000078000000000000000000000000000000000000000000000000F8FDDD
:42A7100008000000000000000000000000000000000000000000000000000000000000000000000000000008080000000000000000000000000000000000000000000080ADFFC3
:42A7520000000000000000000000000000000000000000000000000000000000000000000000000000000000000000000000000000000000000000000000000000000080B4FE93
:42A7940000000000000000000000000000000000000000000000000000000000000000000000000000000078000000000000000000000000000000000000000000000000DAFF32
:42A7D600040000000000000000000000000000000000000000000000000000000000000000000000000000000000000000000000000000000000000000000000000000006DFFD1
:42A8180000000000000000000000000000000000000000000000000000000000000000000000000000000068000000000000000000000000000000000000000000000000F8FCA2
:42A85A00000000000000000000000000000000000000C0080100000000000000000000000000000000000000110000000000000000000000000000000000000000000000F8FEEC
:42A89C00000000000000000000000000000000000000000000000000000000000000000000000000000000000000000000000000000000000000000000000000000000003CFE40
:42A8DE00000000000000000000000000000000000000F000000000000000000000000000000000000000007810000000000000000000000000000000000000000000000024FE9E
:42A9200004000000000000000000000000000000000010440000000000000000000000000000000000000068040000000000000000000000000000000000000000000000E9FC4C
:42A962000C0000000000000000000000000000000000000000000000000000000000000000000000000000008200000000000000000000000000000000000000000000005CFCCD
:42A9A400000000000000000000000000000000000000F000000000000000000000000000000000000000007800000000000000000000000000000000000000000000000034FED7
:42A9E6000800000000000000000000000000000000000000000000000000000000000000000000000000000000000000000000000000000000000000000000000000008034FE75
:42AA2800000000000000000000000000000000000000C0000000000000000000000000000000000000000060080000000000000000000000000000000000000000000000BCFC0C
:42AA6A00000000000000000000000000000000000000000000000000000000000000000000000000000000602000000000000000000000000000000000000000000000007AFEB2
:42AAAC00000000000000000000000000000000000000000000000000000000000000000000000000000000000000000000000000000000000000000000000000000000003CFE2E
:42AAEE0000000000000000000000000000000000000000000000000000000000000000000000000000000078400000000000000000000000000000000000000000000000B8FDB9
:42AB30000800000000000000000000000000000000000000000000000000000000000000000000000000000802000000000000000000000000000000000000000000008085FDCF
:42AB720000000000000000000000000000000000000000000000000000000000000000000000000000000000000000000000000000000000000000000000000000000080B4FE6F
:42ABB40000000000000000000000000000000000000000000000000000000000000000000000000000000078000000000000000000000000000000000000000000000000DAFF0E
:42ABF600040000000000000000000000000000000000000000000000000000000000000000000000000000000000000000000000000000000000000000000000000000006DFFAD
:42AC38000000000000000000000000000000000000000000000000000000000000000000000000000000006000000000000000000000000000000000000000000000000078FC06
:42AC7A00000000000604000000000000000000000000C0080100000000000000000000000000000000000060200000000000000000000000000000000000000000000000FCFF4A
:42ACBC00000000000000000000000000000000000000000000000000000000000000000000000000000000000000000000000000000000000000000000000000000000003CFE1C
:42ACFE00000000800700000000000000000000000000F0000000000000000000000000000000000000000078200000000000000000000000000000000000000000000000A8FD60
:42AD400008000080000200000000000000000000000010400000000000000000000000000000000000000008000000000000000000000000000000000000000000000000E5FC0E
:42AD8200000000000000000000000000000000000000000000000000000000000000000000000000000000000000000000000000000000000000000000000000000000003CFE55
:42ADC400000000800700000000000000000000000000F000000000000000000000000000000000000000007800000000000000000000000000000000000000000000000088FDD9
:42AE060004000000000000000000000000000000000000000000000000000000000000000000000000000000000000000000000000000000000000000000000000000080F4FE94
:42AE4800000000000600000000000000000000000000C000000000000000000000000000000000000000006000000000000000000000000000000000000000000000000090FE14
:42AE8A0000000000000000000000000000000000000000000000000000000000000000000000000000000008000000000000000000000000000000000000000000000000BCFEC4
:42AECC00000000000000000000000000000000000000000000000000000000000000000000000000000000000000000000000000000000000000000000000000000000003CFE0A
:42AF0E000000000000000000000000000000000000000000000000000000000000000000000000000000006000000000000000000000000000000000000000000000000078FC2D
:42AF50000400000000000000000000000000000000000000000000000000000000000000000000000000006000000000000000000000000000000000000000000000000029FD35
:42AF92000C00000000000000000000000000000000000000000000000000000000000000000000000000006082000000000000000000000000000000000000000000000018FE79
:42AFD40000000000000000000000000000000000000000000000000000000000000000000000000000000078000000000000000000000000000000000000000000000000F8FDCE
:42B016000800000000000000000000000000000000000000000000000000000000000000000000000000006020000000000000000000000000000000000000000000008050FCA4
:42B058000000000000000000000000000000000000000000000000000000000000000000000000000000006002000000000000000000000000000000000000000000000058FEFE
:42B09A0000000000000000000000000000000000000000000000000000000000000000000000000000000008000000000000000000000000000000000000000000000000BCFEB2
:42B0DC00000000000000000000000000000000000000000000000000000000000000000000000000000000000000000000000000000000000000000000000000000000003CFEF8
:42B11E0000000000000000000000000000000000000000000000000000000000000000000000000000000018000000000000000000000000000000000000000000000000BCFF1C
:42B160000C000000000000000000000000000000000000000000000000000000000000000000000000000008000000000000000000000000000000000000000000000080E5FF35
:42B1A2000400000000000000000000000000000000000000000000000000000000000000000000000000006020000000000000000000000000000000000000000000008090FCDB
:42B1E40000000000000000000000000000000000000000000000000000000000000000000000000000000078000000000000000000000000000000000000000000000000F8FDBC
:42B226000C00000000000000000000000000000000000000000000000000000000000000000000000000006000000000000000000000000000000000000000000000008021FDDC
:42B268000000000000000000000000000000000000000000000000000000000000000000000000000000006000000000000000000000000000000000000000000000000078FCD0
:42B2AA00000000000604000000000000000000000000C0080100000000000000000000000000000000000000200000000000000000000000000000000000000000000000B8FDBA
:42B2EC00000000000000000000000000000000000000000000000000000000000000000000000000000000000000000000000000000000000000000000000000000000003CFEE6
:42B32E00000000800700000000000000000000000000F04000000000000000000000000000000000000000180000000000000000000000000000000000000000000000008CFF83
:42B370000800008020020000000000000000000000001000000000000000000000000000000000000000000800000000000000000000000000000000000000000000000085FC58
:42B3B200000000000000000000000000000000000000000000000000000000000000000000000000000000600400000000000000000000000000000000000000000000007CFC7D
:42B3F400000000800700000000000000000000000000F000000000000000000000000000000000000000007810000000000000000000000000000000000000000000000098FD83
:42B4360004000000000000000000000000000000000000000000000000000000000000000000000000000060000000000000000000000000000000000000000000000080B0FC44
:42B47800000000000600000000000000000000000000C000000000000000000000000000000000000000006000000000000000000000000000000000000000000000000090FEDE
:42B4BA00000000000000000000000000000000000000000000000000000000000000000000000000000000000000000000000000000000000000000000000000000000001EFC36
:42B4FC0020000480001000024000080001200004800010000240000800012000040000000000100002400000000120000480001000024000080001200004800010000200B4FC34
:42B53E000000000000000000000000000000000000000000000000000000000000000000000000000000004000000000000000000000000000000000000000000000000078FE15
:42B580002C0004800010000240000800012000048000100002400008000120000400000000001000024000080001200004800010000240000800012000048000100002806DFD61
:42B5C20004000000000000000000000000000000000000000000000000000000000000000000000000000000000000000000000000000000000000000000000000000080F4FED1
:42B60400200004000010000240000800012000048000000002400008000120000400000000001000024000000001200004800010000240000800012000048000100002003CFD31
:42B646000C000000040000000000000000000000000080000000000000000000000000000000000000000040000000000000000000000000000000000000000000000080ADFFC6
:42B688002000048000100002400008000120000480001000024000080001200004000000000010000240000800012000048000100002400008000120000480001000020034FC1E
:42B6CA00000000000000000000000000000000000000000000000000000000000000000000000000000000000000000000000000000000000000000000000000000000003CFE04
:42B70C00000000000000000000000000000000000000000000000000000000000000000000000000000000000000000000000000000000000000000000000000000000003CFEC1
:42B74E00000000000000000000000000000000000000000000000000000000000000000000000000000000000000000000000000000000000000000000000000000000003CFE7F
:42B79000000000000000000000000000000000000000000000000000000000000000000000000000000000000000000000000000000000000000000000000000000000003CFE3D
:42B7D200000000000000000000000000000000000000000000000000000000000000000000000000000000000000000000000000000000000000000000000000000000003CFEFB
:42B81400000000000000000000000000000000000000008000000000000000000000000000000000000000002000000000000000000000000000000000000000000000009CFEB8
:42B856000000000000000000000000000000000000000000000000000000000000000000000000000000000800000000000000000000000000000000000000000000008016FC16
:42B89800000000000000000000000000000000000000000000000000000000000000000000000000000000000000000000000000000000000000000000000000000000003CFE34
:42B8DA00000000000000000000000000000000000000000000000000000000000000000000000000000000000000000000000000000000000000000000000000000000003CFEF2
:42B91C00000000000000000000000000000000000000000000000000000000000000000000000000000000000000000000000000000000000000000000000000000000003CFEAF
:42B95E00000000000000000000000000000000000000000000000000000000000000000000000000000000000100000000000000000000000000000000000000000000002CFF7B
:42B9A0000000000000000000000000000000000000000000000000000000000000000000000000000000000000000000000000000000000000000000000000000000008096FC53
:42B9E200000000000000000000000000000000000000000000000000000000000000000000000000000000201000000000000000000000000000000000000000000000002CFCCB
:42BA2400000000000000000000000000000000000000000000000000000000000000000000000000000000000000000000000000000000000000000000000000000000003CFEA6
:42BA6600000000000000000000000000000000000002000000000000000000000000000000000000000000102000000000000000000000000000000000000000000000001CFD53
:42BAA80000000000048000000000000000000000009400000000000000000000000000000000000000000000000000000000800000000000000000000000000000000000ECFFD9
:42BAEA00000000000000000000000000000000000000000000000000000000000000000000000000000000000000000000000000000000000000000000000000000000003CFEE0
:42BB2C0000000000048000000000000000000000000404000000000000000000000000000000000000000000000000000000800000000000000000000000000000000000B4FE19
:42BB6E00000000000000000000000000000000000000000000000000000000000000000000000000000000000000000000000000000000000000000000000000000000003CFE5B
:42BBB000000000000000000000000000000000000000000000000000000000000000000000000000000000100000000000000000000000000000000000000000000000003CFF08
:42BBF200000000000000000000000000000000000000000000000000000000000000000000000000000000000000000000000000000000000000000000000000000000003CFED7
:42BC3400000000000000000000000000000000000000000000000000000000000000000000000000000000000000000000000000000000000000000000000000000000003CFE94
:42BC7600000000000000000000000000000000000000000000000000000000000000000000000000000000000000000000000000000000000000000000000000000000003CFE52
:42BCB800000000000000000000000000000000000000000000000000000000000000000000000000000000000000000000000000000000000000000000000000000000003CFE10
:42BCFA00000000000000000000000000000000000000000000000000000000000000000000000000000000000000000000000000000000000000000000000000000000003CFECE
:42BD3C00000000000000000000000000000000000000000000000000000000000000000000000000000000000000000000000000000000000000000000000000000000003CFE8B
:42BD7E00000000000000000000000000000000000000000000000000000000000000000000000000000000000000000000000000000000000000000000000000000000003CFE49
:42BDC000000000000000000000000000000000000000000000000000000000000000000000000000000000000000000000000000000000000000000000000000000000003CFE07
:42BE0200000000000000000000000000000000000000000000000000000000000000000000000000000000000000000000000000000000000000000000000000000000003CFEC4
:42BE4400000000000000000000000000000000000000000000000000000000000000000000000000000000000000000000000000000000000000000000000000000000003CFE82
:42BE86000000000008000000000000000000000000000001000000000000000000000000000000000000000000000000000000000000000000000000000000000000000024FF4E
:42BEC8000000000008000000000000000000000000000001000000000000000000000000000000000000000000000000000000000000000000000000000000000000000024FF0C
:42BF0A00000000000000000000000000000000000000000000000000000000000000000000000000000000104000000000000000000000000000000000000000000000007CFF2A
:42BF4C0000000000000000000000000000000000000020000000000000000000000000000000000000000000800000000000000000000000000000000000000000000000BCFC5B
:42BF8E00000000001000000000000000000000000000000000000000000000000000000000000000000000000000000000000000000000000000000000000000000000002CFE37
:42BFD000000000000000000000000000000000000000000000000000000000000000000000000000000000000000000000000000000000000000000000000000000000003CFEF5
:42C012000000000000000000000000000001000000000000000000000000000000000000000000000002000000000000000080000000000000000000000000000000008026FFC4
:42C05400000000000000000000000000000000000000000000000000000000000000000000000000000000000000000000000000000000000000000000000000000000003CFE70
:42C096000000000000000000000000000004000000000100000000000000000000000000000000000008010000000000000000020000000000000000000000000000000020FD3B
:42C0D800000000800020010000000000000000000020200000000000000000000000000000000000000008102000000000008000000000000000000000000000010000009CFDF3
:42C11A00000000000000000000000000000000000000000000000000000000000000000000000000000000000000000000000000000000000000000000000000020000001CFEC7
:42C15C0000000000000000000000000000000000000000000000000000000000000000000000000000000000000000000000800000000000000000000000000000000000BCFE67
:42C19E00000000000000000000000000000000000000000000000000000000000000000000000000000000000000000000000000000000000000000000000000000000003CFE25
:42C1E000000000000000000000000000000000000000000000000000000000000000000000000000000000000000000000000000000000000000000000000000000000003CFEE3
:42C22200000000000000000000000000000000000000000000000000000000000000000000000000000000000000000000000000000000000000000000000000000000003CFEA0
:42C26400000000000000000000000000000000000000000000000000000000000000000000000000000000000000000000000000000000000000000000000000000000003CFE5E
:42C2A600000000000000000000000000000000000000000000000000000000000000000000000000000000000000000000000000000000000000000000000000000000003CFE1C
:42C2E800000000000000000000000000000000000000000000000000000000000000000000000000000000000000000000000000000000000000000000000000000000003CFEDA
:42C32A00000000000000000000000000000000000000000000000000000000000000000000000000000000000000000000000000000000000000000000000000000000003CFE97
:42C36C00000000000000000000000000000000000000000000000000000000000000000000000000000000000000000000000000000000000000000000000000000000003CFE55
:42C3AE00000000000000000000000000000000000000000000000000000000000000000000000000000000000000000000000000000000000000000000000000000000003CFE13
:42C3F000000000000000000000000000000000000000000000000000000000000000000000000000000000000000000000000000000000000000000000000000000000003CFED1
:42C43200000000000000000000000000000000000000000000000000000000000000000000000000000000000000000000000000000000000000000000000000000000003CFE8E
:42C47400000000000000000000000000000000000000000000000000000000000000000000000000000000000000000000000000000000000000000000000000000000003CFE4C
:42C4B60080040000000000000000000000000000000000000000000000000000000000000000000000000000000000000000000000000000000000000000000000000000B0FE12
:42C4F800000100000000000000000000000000000000000000000000000000000000000000000000000000000000000000000000000000000000000000000000000000002CFFD6
:42C53A00000000000000000000000000000000000000000000000000000000000000000000000000000000000000000000000000000000000000000000000000000000003CFE85
:42C57C00000000000000000000000000000000000000000000000000000000000000000000000000000000000000000000000000000000000000000000000000000000003CFE43
:42C5BE000017E002A8000950012A4005A8002DA0025C800B50012A4005A80015400200000000000950012A4005F80115A00254800A50012A800450011240054800092001E8FC60
:42C60000800C9001100106880011200244804010013240068800112002448008800100000000000688001120026482081001224004880011000320020C8008300006C00060FCAA
:02C64200FFFFF8
:00000001FF
